:020000040000FA
:1000000001282100F030990020008C0122008C0191
:1000100023008C012100A7309500210038308C008E
:1000200020008B01A001A101A201A301A401BF2016
:10003000BF200030A9000030AA00C330AB00503010
:10004000AC002300910184201308F00084201308E1
:10005000F10084201308F20084201308F30020002C
:100060002C08B4002B08B5002A08B6002908B700F0
:10007000A801A701A601A5018820BF208830A500FE
:100080001330A60047205F208820BF204228250883
:10009000B407031C5028B50F5028B60F5028B70AD4
:1000A0002608B507031C5728B60F5728B70A270894
:1000B000B607031C5C28B70A2808B7070800FE30FB
:1000C000370703187B2801303702031C8328D230FE
:1000D000360703187B282D303602031C832839305D
:1000E000350703187B28C6303502031C8328C0302F
:1000F0003402031C83282C08B4002B08B5002A08FE
:10010000B6002908B700080015141308910A080062
:10011000A001A101A201A301A4012030AD0070083B
:10012000B0007108B1007208B2007308B300031088
:10013000301CB1283408A107031CA328A20FA32850
:10014000A30FA328A40A3508A207031CAA28A30FFB
:10015000AA28A40A3608A307031CAF28A40A370854
:10016000A407A40CA30CA20CA10CA00CB30CB20C01
:10017000B10CB00CAD0B97280030A4000800203063
:10018000860000308700403FAF000830AE00AF0C63
:10019000031CD0280C1400000C1500000C11D528ED
:1001A0000C1000000C1500000C11AE0BC728860ABD
:1001B00025300602031CC3288C1400008C1000009C
:0801C0000C1000000C110800F6
:020000040001F9
:02000E00A40943
:02001000FF1CD3
:08E00000D00017005C002200B3
:00000001FF
